:020000040000FA
:1000000001288B018316031300309B008113FE30FF
:100010008600831203130730900022140E1C221056
:1000200014202F201F200D2822080139A000831240
:1000300003175D088312031320068600080015309D
:10004000A10000000000000000000000000000000F
:10005000A10B212800000000000000000800031090
:10006000A20DA30DA40DA50DA60DA70DA80DA90DFC
:10007000AA0DAB0DAC0DAD0DAE0DAF0DB00DB10DAC
:10008000B20DB30DB40DB50DB60DB70DB80DB90D5C
:10009000BA0DBB0DBC0DBD0DBE0DBF0DC00DC10D0C
:1000A000C20DC30DC40DC50DC60DC70DC80DC90DBC
:1000B000CA0DCB0DCC0DCD0DCE0DCF0DD00DD10D6C
:1000C000D20DD30DD40DD50DD60DD70DD80DD90D1C
:1000D000DA0DDB0DDC0DDD0DDE0DDF0DE00DE10DCC
:1000E000E20DE30DE40DE50DE60DE70DE80DE90D7C
:1000F000EA0DEB0DEC0DED0DEE0DEF0DF00DF10D2C
:10010000F20DF30DF40DF50DF60DF70DF80DF90DDB
:10011000FA0DFB0DFC0DFD0DFE0DFF0D83160313F7
:10012000A00DA10DA20DA30DA40DA50DA60DA70D4B
:10013000A80DA90DAA0DAB0DAC0DAD0DAE0DAF0DFB
:10014000B00DB10DB20DB30DB40DB50DB60DB70DAB
:10015000B80DB90DBA0DBB0DBC0DBD0DBE0DBF0D5B
:10016000C00DC10DC20DC30DC40DC50DC60DC70D0B
:10017000C80DC90DCA0DCB0DCC0DCD0DCE0DCF0DBB
:10018000D00DD10DD20DD30DD40DD50DD60DD70D6B
:10019000D80DD90DDA0DDB0DDC0DDD0DDE0DDF0D1B
:1001A000E00DE10DE20DE30DE40DE50DE60DE70DCB
:1001B000E80DE90DEA0DEB0DEC0DED0DEE0D8312E2
:1001C0000317900D910D920D930D940D950D960DB5
:1001D000970D980D990D9A0D9B0D9C0D9D0D9E0DE3
:1001E0009F0DA00DA10DA20DA30DA40DA50DA60D93
:1001F000A70DA80DA90DAA0DAB0DAC0DAD0DAE0D43
:10020000AF0DB00DB10DB20DB30DB40DB50DB60DF2
:10021000B70DB80DB90DBA0DBB0DBC0DBD0DBE0DA2
:10022000BF0DC00DC10DC20DC30DC40DC50DC60D52
:10023000C70DC80DC90DCA0DCB0DCC0DCD0DCE0D02
:10024000CF0DD00DD10DD20DD30DD40DD50DD60DB2
:10025000D70DD80DD90DDA0DDB0DDC0DDD0D8312B8
:04026000031308007C
:02400E00223F4F
:02401000FC3F73
:00000001FF
